:0300000002106883
:0C10680078FFE4F6D8FD7581DA0210AFC5
:01003A0022A3
:061A37008B528A53895412
:101A3D007576027F48121B75121D7AEF20E0F9AB07
:101A4D0052AA53A954120858787CE6FE08E6FDED1B
:011A5D00FF89
:011A5E002265
:100E5400434647002D53322D0052415445434C52D2
:100E640020554E49544C49544554524947545245CF
:100E7400565354525453544F505A4355545A543160
:100E8400205A5432205A45524F4241554444464C0C
:100E9400545341564552535420504320205F31202F
:100EA400735F3220735F35207331207320322073D7
:100EB4002035207320313020733330207331206D7E
:100EC4002032206D2035206D203130206D333020CC
:100ED4006D312068200000000100020005000A00B6
:100EE4001400320064012C025804B00BB817704689
:100EF400508CA00102040810304665657459617273
:100F0400644D6574724F6666204F6E20204E6F20CC
:100F140020596573204F6666204F666620547269B7
:100F2400674F6666205472696753747274526563BE
:010F3400209C
:10159400740526F618E436F6C308E62225E024D9B5
:1015A400F582E4340EF58322900EF79375F018A4B7
:1015B400FFAEF0220554E554C39403220554E554C8
:1015C400C3940222A654E55475F004A42208F60834
:0415D400F608F622FD
:10165F00789C76AB0876CD08760008760AE408F613
:10166F0008760108F60876640876401215D108F658
:10167F0078AAF608761E08F608763C0876010876F2
:10168F005E0876010876901215D178B776050219A3
:01169F00E466
:10195A00751E1D751FC0121502789DE664CD7004B0
:10196A0018E664AB600312165F78B6E6FFF460030C
:0F197A00EF700478B6760478B7E6B4FF0276050E
:01198900223B
:101C1F00C2AF5387DF7DC07C1DE4FF121C47438793
:031C2F0020D2AF11
:011C3200228F
:10150200755FFF851E60851F6175620075630075DA
:10151200649CE4FFAB5FAA60A9618F8275830012AD
:10152200082BAB62AA63A9648F8275830012086AD2
:101532000FBF1CE078B5E6FFF46003EF700478B5E6
:0A154200760478B6E6B401027604E0
:01154C00227C
:1019E4007D01E4FF121B3A121C1FC2AF5387DF7F35
:1019F4009C7B1C7DC07C1D121C51438720D2AF7F71
:0A1A040002121889E4FDFF021B3AEC
:10030B00E4F5527BFF7A0E79541217637F051218AE
:10031B0089A297829650FAA2969215A2979216E509
:10032B005275F004A4245DF9740E35F0FA7BFF12BC
:10033B0017637F05121889855253E4F5547BFF7AB6
:10034B000E7958121763E552B40D0040030203F9FE
:10035B00900362F82828730203890203F90203AAA7
:10036B000203B20203B60203BE0203C60203CA02B1
:10037B0003DA0203DE0203E20203D20203EE7F0181
:10038B00EF1215A0789EE6FC08E6FD7401936D70E4
:10039B0003E4936C70028F540FBF0FE40204887850
:1003AB00A0E6F5540204A778A1800278A9E6F554DB
:1003BB000204C178A8E6F5540204F078B280027802
:1003CB00B3E6F55402050A78B4E6F55402059178C4
:1003DB00B0800678AA800278ACE6FE08E6FFF554FA
:1003EB000205BA78B7E6F5541215AC0205BAE55218
:1003FB006553600302032AA215309601B35013A272
:10040B0096921530960C0552E552C394104003E4B6
:10041B00F552A216309701B350D4A297921630978B
:10042B00CDE552B4100050C690043AF82828730258
:10043B00046A0204930204990204B30204CD020479
:10044B00E20204FC02051602052B020549020564B3
:10045B0002057F0205A50205C00205C60205CC05F3
:10046B0054E554C3940F4003755401E5541215A081
:10047B00E493FF740193789ECFF608EFF61215CA3A
:10048B00249DF9740E02059A1213B90203F9121581
:10049B00B84003E4F55478A0A654E55475F004A4D1
:1004AB0024FDF9740E02059A1215C04003E4F554AD
:1004BB0078A1A654E55475F004A42409F9740F022D
:1004CB00059A1215C04003E4F55478A91215C824F7
:1004DB0009F9740F02059A1215C04003E4F554781C
:1004EB00A8A654E55475F004A42411F9740F020561
:1004FB009A1215B84003E4F55478B2A654E5547536
:10050B00F004A42419F9740F02059A1215B84003CC
:10051B00E4F55478B31215C82419F9740F02059A2F
:10052B0078B1743212159694DC18E6940540057672
:10053B000008766478B0E6FE08E6FF0205BA78ABF1
:10054B00121594942C18E694014005760008760A4F
:10055B0078AAE6FE08E6FF805678AD121594942C27
:10056B0018E694014005760008760A78ACE6FE089A
:10057B00E6FF803B0554E554C394044003E4F55473
:10058B0078B4A654E55475F004A42425F9740F35FA
:10059B00F0FA7BFF1217630203F90554E554C39479
:1005AB00064003E4F55478B7A654E5541215AC1283
:1005BB0012740203F912165F0203F91219E4020313
:0705CB00F943A2080203F945
:0A1D56004552415300444F4E450032
:101CD100789EE6F52E08E6F52F22E50BAE0A78068A
:011CE10022E0
:1010F400C213C21478B6E6FFE4FCFDFEFB7A20F9C5
:10110400F812088C8F118E108D0F8C0EE47B40FA30
:10111400F9F81209178E088F09E4F553F554C3E55D
:10112400549509E5539508501CE55264816016AF47
:1011340054AE5312198A121C338F520554E554705D
:10114400DD055380D9E552B48108E5541554700285
:101154001553E55465097004E5536508700CD21302
:10116400121D21E4F50AF50B800785530A85540BFB
:0B117400E4F50CF50D752D80121CD168
:01117F00224D
:10198A00C3EF9509EE95085024EF7806C333CE339A
:10199A00CED8F9FD757602EE787CF6CFEDCFEF085A
:0D19AA00F67F50121BDE121D7AEF20E0F9CF
:0119B700220D
:031BAB00CDEFCDAE
:101BAE00757602EE787CF6ED08F67F50121BDE128B
:061BBE001D7AEF20E0F9A2
:011BC40022FE
:101C33007576017F50121B75121D7AEF20E0F9783B
:031C43007CE6FF3D
:011C4600227B
:101BF500121BABE4FFFE0FBF00010EBE0FF8BFA026
:041C0500F5121C3385
:011C090022B8
:0618BF00CBEFCBCAEECA1C
:1018C500301303301427757603EA787CF6EB08F6B7
:1018D50008EDF67F50121BDE121D7AEF20E0F9E4C9
:0D18E500FFFE0FBF00010EBE0FF8BFA0F503
:0118F20022D3
:1016A00075550075560075572DE4F554121CDBC3B3
:1016B00033CE33CED8F97C002554FFEC3EFEAB553B
:1016C000AA56A95785548275830012082BFD12185B
:1016D000BF0554E554C3940640D2750C00750D0641
:0116E00022E7
:1011FC008E528F53121CDBC333CE33CED8F9250D50
:10120C00FFE50C3EFEEEC0E0EFC0E0E552FDD0E0A5
:10121C00FFD0E0FE1218BF050DE50D7002050C1293
:10122C001CDBC333CE33CED8F9250DFFE50C3EFEC7
:10123C00AD531218BF050DE50D7002050C0531E517
:10124C003170020530C3E50D9440E50C9400401755
:10125C00E4F50CF50D050BE50B7002050A9509E597
:08126C000A95084002D213228A
:1013B900E4F50CF50D7BFF7A1D7956121763D214EB
:1013C900E4F55FF560C3E5609509E55F950850218F
:1013D900E560AE5F7806C333CE33CED8F9F50D8E0E
:1013E9000C7D81FF1218BF0560E56070D8055F802C
:1013F900D4C2147BFF7A1D795B121763E4F50AF5F1
:071409000BF50CF50DC213F9
:0114100022B9
:10136000E4F55FF560F561F562C3E5629509E56155
:1013700095085044E5606481603EAF62AE61121929
:101380008A121C338F60E56064807022AF5F055F56
:10139000FCFDFEFBFAF9120A187F2C121D80AE61CB
:1013A000AF62E4FCFDFBFAF9120A18121D6A05622D
:0813B000E56270B5056180B132
:0113B8002212
:02154D008F5FAE
:10154F00E4F560F561F562F563C3E5639509E5625E
:10155F0095085030E5616481602AAF63AE6212195D
:10156F008A121C338F61E561B4800FE560655F708F
:10157F0007AF63AE6202198A05600563E56370C940
:04158F00056280C5AC
:011593002235
:1016E100121CD178A9E6F532E4F530F5311216A0D5
:1016F100850A12850B137F01121AAD30021A78ACDC
:10170100E6FE08E6FFE4FCFD7B64FAF9F812088CBA
:101711008F4C8E4B8D4A8C49300505C205121D3DFB
:0117210022A5
:1017E000850A52850B53E50D450C60080553E553FA
:1017F0007002055285120A85130B1216A085520A33
:1018000085530BC3E5539509E55295084007E4F568
:0A1810000AF50BD2137F02021AAD95
:101C4700740478FF769612FF0322740078FF769665
:041C570012FF032253
:03003300020D615A
:100D6100C0E0C0F0C083C082C0D0E8C0E0E9C0E00C
:100D7100EAC0E0EBC0E0ECC0E0EDC0E0EEC0E0EFC7
:020D8100C0E0D0
:100D8300E5D954F8FF1209F20DB0080DB0100DBFEC
:100D9300180DDA200DC1280DDA300DDC380DE240D4
:100DA3000DDA480DFB500E185800000E268579DA2F
:100DB300C2DDC2DC7577007578008070800EE57641
:100DC300700280560578E5787002057712000E8F61
:100DD300DAC2DDC2DC80558016D2DDC2DC804DC2B2
:100DE300DDC2DCE5767004C2DA8041D2DA803DC22E
:100DF300DDD2DC7574048034AFDA121D4A0578E560
:100E03007870020577C2DDC2DCE5767004C2DA8051
:100E13001BD2DA8017AFDA121D4AC2DDD2DC757439
:0E0E2300028009757404C2DDC2DCD2DAC2DBC3
:100E3100D0E0FFD0E0FED0E0FDD0E0FCD0E0FBD080
:100E4100E0FAD0E0F9D0E0F8D0D0D082D083D0F071
:030E5100D0E032BC
:1019B80043910C43920CE4F5DBEF25E0F5DB3015A1
:1019C8000343DB0175DD1775DC1775D84453F8FE42
:0C19D80053F7FE43F701E4F574D2E82257
:101BDE00E57430E002FF22E4F575757403EF25E03D
:071BEE00F579D2DD7F022230
:101B7500E57430E002FF22E4F5751576757405EF1E
:0B1B850025E04401F579D2DD7F02224B
:061D7A0020DBFDAF742226
:0D000E001576AF750575747C2FF8E6FF229E
:0C1D4A00747C2575F8EFF60575157622FF
:0D0026007584C075853F53913F759200228F
:1017A300C3E49515F517E49514F51622C3E51595CD
:1017B3002BF51AE514952AF51922E52B9515F51A3B
:1017C300E52A9514F51922C3E4952BF517E4952A18
:0D17D300F51622D3E52B9515E52A95142275
:101AF900E4F593758640F5944384405385BF53F8C4
:101B0900FD53F7FD43F80243F702F518C20CD2E979
:011B190022A9
:03003B00020B3F76
:100B3F00C0E0C0D0E8C0E0EDC0E0EEC0E0EFC0E044
:100B4F00308610C20C758D00758B00D28E75940295
:100B5F00020C43C28EAF8DEFAD8BF514EDF515057D
:100B6F0018E548146034146057147003020C001415
:100B7F007003020C13147003020C3224056003027D
:100B8F000C351217A3E518C394645003020C358576
:100B9F00142A85152B0548020C351217A31217D6E8
:100BAF0040051217BD80031217AFD3E51A94E1E584
:100BBF001994024071753A00753B000548020C35D7
:100BCF001217A3C3E53B78AB96E53A189650167803
:100BDF00B0E6FE08E6FFC3E5349FEE6480F8E53328
:100BEF0064809840417528007529000548D20D8012
:100BFF00351217CAC3E52978AD96E5281896402611
:100C0F00054880221217CA1217D640051217BD8049
:100C1F00031217AFC3E51A94B8E5199400500705EE
:100C2F004880031217A3E516F58D85178BD287D24F
:100C3F008E7594005394FED0E0FFD0E0FED0E0FD1F
:080C4F00D0E0F8D0D0D0E03273
:1012EC00AF2BAE2A121350AF15AE14121350AF170A
:1012FC00AE16121359AF48121BC57F20121D80AFBA
:10130C0034AE33121CE27F20121D8078B0E6FE084A
:10131C00E6FF12135978AA121342AF3BAE3A121CD5
:10132C00E2121D6A78AC121342AF29AE28121CE2ED
:10133C00121D6A021D6AE6FE08E6FF121CE27F20FF
:10134C00121D8022121CE27F20121D8022121CE230
:04135C00121D6A22D2
:101A86006F035D5733767E437F771004007B3E6C91
:101A96001F7C78773B020F382C5A1A6F79751876A7
:071AA6003C0E2F4E2B375DB3
:101927004EFECCEFCC0F747C2CF8EEF6EDC43322D0
:10193700901A92E493FF78D0F608EFF608F608F6C7
:1019470022E493FF74D02EF8EFF60E22EE3395E0E3
:03195700FDFC2272
:100FD500E4FF0F247CF876CD0F747C2401F876802D
:100FE5000F747C2402F876E00F747C2403F876F8FD
:100FF50030170A0F747C2404F87671800ACEEFCE80
:101005000F747C2EF8767078D0E6FEC4540FFDCCB4
:10101500EFCC0F747C2CF8EDF6EEC454F0FE78D1CD
:10102500E6FD131313541F12192754E0FE78D2E678
:10103500FD1313543F1219273354C0FE78D3E6FD30
:10104500C31312192733335480FECDEFCD0F747CB3
:101055002DF8EEF68F767F38121BDE121D7AEF2003
:02106500E0F9B0
:011067002266
:1018F300C21712193775760A787C76CD0876800878
:1019030076E00876F80876700876050876D50876C6
:101913009B0876FFE408F67F38121BDE121D7AEF70
:0319230020E0F9C8
:01192600229E
:101B9000EF24F9600B14600C2402700EC21780074A
:0B1BA000D2178003121937120FD52254
:10141100C3EF648094E1400ED3EF648094FA5006E8
:10142100EF24ACFF803CC3EF648094C1400ED3EF46
:10143100648094DA5006EF24CCFF8026C3EF6480E9
:1014410094B0400ED3EF648094B9500674D02FFF4E
:101451008010BF2D047F0A8009BF5F047F0B8002CB
:031461007F0C22DB
:101A5F00CEEDCECDEFCDCFEECF121411EF3395E00B
:101A6F00FE74862FF582741A3EF583E493FF74D0CB
:071A7F002DF8EFF6020FD570
:061763008B618A628963BC
:10176900E4FE901A92121948BE04F7E4FEAB61AA8E
:1017790062A9638E8275830012082BFF6019121407
:1017890011EFFD3395E0FC74862DF582741A3CF552
:0A17990083121948BE04D6020FD5D2
:041274008F828E8354
:101278001219537B197AFC79FF78FFD31209B7400A
:101288000390FC19AF82AE83121953E47B0F7A27BF
:10129800F9F8C31209B7500390270FE4F55574CB3A
:1012A8002555F8E4F60555E555B405F2AE83AF8249
:1012B8001219537B007A0079CB120A1878CEE6709F
:1012C8001A75550374CA2555F8E6FF74CB2555F8E9
:1012D800EFF6D555EF78CB762080E17B007A007960
:0412E800CB021763BB
:101CAB00C210C212C20FE4FDFF121B3AE4FD7F010A
:031CBB00021B3ACF
:101B3A00EF146011047016BD0104C2828002D282C1
:0E1B4A00A282921122BD0103C28122D2812209
:101AAD00EF24FE600D14601124027019D210751C04
:101ABD000122C210A211928222D212751D027D0145
:061ACD007F01121B3A220A
:101A0E00301012D51C0F308207C282751C0F800554
:101A1E00D282751C23E51DD39400400CD51D09C23E
:091A2E0012E4FD7F01121B3A22B3
:0F1D120046554C4C005A46354A0020342D3200BD
:030036000135632E
:101C0A00F543F542F541F540853F27853E26853D5A
:051C1A0025853C242299
:021889008F606E
:10188B00E4F561F562C3E5629560E5619400502370
:10189B00900000AF82AE83E4FCFD7B207A4EF9F81A
:1018AB00D31209B74003A380EA0562E56270D6053F
:0318BB006180D277
:0118BE002207
:0E1D21007BFF7A1D79121217637F0A02188960
:0F1D0300D20B301306121D21C20B221216E12241
:05001E00C20B0217E017
:0D1D3D00E4121C0AF53FF53EF53DF53C2291
:101CF3008E7A8F7BEEFF121D80AF7BE57B021D800A
:10003E00120026121D60121CAB7F04121889209725
:10004E000B7D057F01121180D2AF80FE209612D259
:10005E00AF12195AC2157F701219B81210F412038A
:10006E000B12195A78B7E6FDE4FF12118043872070
:10007E00D2AFC2157F701219B87F011218891210F3
:10008E00F41218F37A1D79171203007A1D791C12D7
:10009E00030012003AE478DAF61217227F011218E2
:1000AE0089121D83A2969208A2979209E4F54DF546
:1000BE0039F538F537F536F54E7543F17542D87585
:1000CE0041FF7540FFF527F526F525F524C20AF503
:1000DE003FF53EF53DF53CC20BF54FF550C20DF523
:1000EE002078A1E66004D2808002C28078B4E62433
:1000FE00FE600B14600C2402700AD2038006D20438
:10010E008002D205E4F548752C64121AF978DAE605
:10011E00C3940240F8E4F6D52C13752C64053BE528
:10012E003B7002053A0529E529700205282096053F
:10013E00209702D20E30963030972D300E2AC20EF6
:10014E00AF27AE26AD25AC24EC4D4E4F7005121CDC
:10015E000A8011E4F543F542F541F540F527F52601
:10016E00F525F524D209D208A208309601B3501A0B
:10017E00A2969208309613200E10300A06C20A7FFD
:10018E00068004D20A7F07121B90A209309701B392
:10019E005017A2979209309710200E0DB20B300B0C
:1001AE0005121D03800312001E1205D2054EE54EE8
:1001BE00C3940150030202EEE4F54EFB7A0079512E
:1001CE00121A3778D4EEF608EFF6E55164026003A2
:1001DE000202EE78D4E6FE08E6FF78A0E6FD1214E1
:1001EE00B6E5392FF539E5383EF538E5373DF537C3
:1001FE00E5363CF536054DE54DC394055003020238
:10020E00EEAF39AE38AD37AC36E47B05FAF9F812FD
:10021E0015D88F398E388D378C36C3E5399527F53D
:10022E0039E5389526F538E5379525F537E53695D0
:10023E0024F536AF43AE42AD41AC40AB39AA38A936
:10024E0037F8D31209B7400C8539438538428537C4
:10025E0041853640300A0AAF4378D6E542F608EFBC
:10026E00F6AE38AF3978D4EEF6FE08EFF68E33F5EB
:10027E0034300A0308800278D4E6FE08E6FF121234
:10028E00740550E5507002054FC3789F96E54F18E0
:10029E0096402EE4F54FF550300B267F03121AAD23
:1002AE00201318300D097F007E821211FCC20D78CA
:1002BE00D4E6FE08E6FF1211FC8006121D21120084
:1002CE001E85393F85383E85373D85363CE4F53908
:1002DE00F538F537F536F54D300405C204121D3DDF
:1002EE00E535654860068548351212EC121A0E0285
:0202FE00011BE2
:0B0300007BFF1217637F041218892294
:101AD300444C0021536967005A46354A004D4F4430
:101AE30000342D32004A756E2032332032303037C5
:061AF3000050524F4700B5
:10161C00AF5AAE59AD58AC57EC4D4E4F22EF24FF9C
:10162C00F55AEE34FFF559ED34FFF558EC34FFF56F
:10163C005722E4755A2075594EF558F55722E47522
:10164C005A01F559F558F557227554007555007522
:03165C00569C2277
:1005D200121D2FEF70030207F2121B58EF1209F2DD
:1005E20007CB2407D62A07C04D07DB50071852064F
:1005F2000D61069D6307EF6406F37206F073071C34
:1006020074079076078B78000007F2C20A7BFF7AA4
:100612001A79D312176312163E121D2FEF700A12A7
:10062200161C600512162980F012161C70030207B0
:10063200F2121B588F5312154DE4F55A12164EE45E
:100642007F06FEFDFCAB5AAA59A958A857C3120946
:10065200CD501F121C338F53121D80E55A2401F511
:100662005AE43559F559E43558F558E43557F557F4
:1006720080CD121C338F53E55364806016E55364BA
:10068200816010121D80121C338F53121D8075520F
:10069200018003E4F552E55270D822121655121663
:1006A2004AF55312161C602412163E121D2FEF70CB
:1006B2000A12161C600512162980F012161C60031D
:1006C2001207F30553E553C3941C40D712161C605E
:1006D2001A789CB6AB0708B6CD030207D37BFF7A24
:1006E2001A79D61217637F0A021889020788021341
:1006F20060121655E4F553AB540556E556AA5570EB
:1007020002055514F9120812FF121D800553E55314
:10071200C3941C40E22243A20822C20A7554007507
:1007220055007556D812164AF55312161C6024123B
:10073200163E121D2FEF700A12161C6005121629A2
:1007420080F012161C60031207F30553E553C3949D
:100752000240D712161C602E78D8E6FE08E6FFEE9D
:100762003395E0FDFCC3EF953FF55EEE953EF55DFA
:10077200ED953DF55CEC953CF55BAF5E78A6E55DED
:10078200F608EFF6804B021502C20A0213B97A1A72
:1007920079DB1208077A1A79E0121CBE78B5E624D2
:1007A20030FF121D80121D6A7F76121D807A1A791F
:1007B200E41208077A1A79E8121CBE021D6AE4F5EF
:1007C20053435301AF53021D80C20AE478A6F608D0
:1007D200F60219E4C20A02165FC20A7BFF7A1A798C
:1007E200F41217637D017F0112118080FE1212EC58
:1007F20022121B58AB54AA55A95685538275830001
:10080200EF12086A227BFF121CBE121D6A7BFF22B6
:0A1D6000E4F5955396BF53A27F22CD
:101722005389F0438901538FFE758C70E4F58A5317
:10173200B8FD53B7FD43B702D2A9D28C53890F43E8
:101742008910538FEFF58DF58B53847F438580533A
:10175200A2DF53B8F743B80853B7F743B708D2AB81
:011762002264
:03000B00021C5B79
:101C5B00C0E0E8C0E078DA06758C70758A00D0E0D9
:041C6B00F8D0E0329B
:03001B00021D7350
:071D7300C287C28ED20C32C0
:101C6F000D0A00303132333435363738394142437B
:041C7F004445460092
:101C8300AF73AB67AA68A969057322AF66AE65AD8A
:041C930064AC6322B8
:101180005387BF75985053877FE4F5BABF01054375
:10119000A240800353A2BFE4F5BDED1460151460B6
:1011A0001A14601F1460242404702575BEF075BFE6
:1011B0000B802375BEF075BF05801B75BEF075BF33
:1011C00002801375BE7075BF01800B75BEB08003C1
:1011D00075BE30E4F5BF75BD035391FE43920143E4
:1011E00091025392FDC21853B8EF53B7EF43B810B2
:0C11F000E478C9F618F678CAF6D2AC22F2
:030023000218526E
:10185200C0E0C0D0E8C0E030981E78C9E6C3940F5B
:10186200501418E60624B8F8A69978C90618E6C3F3
:10187200941040027600C298309904C299C218D0DE
:07188200E0F8D0D0D0E03205
:080003002018FDD2188F99228C
:101B1A0078C9E6D39400401508E60624B8F8E6FF2B
:0F1B2A0078C91608E6C394104005E4F6227F0040
:011B39002289
:031D80000200035B
:101B58007F207E4E78C9E67010D3EF9400EE940093
:0C1B68004007EF1F70EE1E80EB121B1AEE
:011B7400224E
:101CBE00120812FF600C121D80740129F9E43AFA21
:031CCE0080EE2283
:0E1D2F0078C9E6D3940040037F01227F002292
:101BC500CEEFCEEE54F0C4540F901C7293FF121D4D
:091BD50080EE540F93FF021D8005
:101CE200CDEFCDCCEECCEEFF121BC5CFEDCF021B5C
:011CF200C52C
:091D6A007BFF7A1C796F021CBE9C
:0E0A18008F668E658D648C638B678A68896932
:100A2600E4F573EC4D4E4F7017E94A4B70057F3075
:100A3600021D80121C838F827583007430020B3B6B
:100A4600121C90EC33502AE5694568456770077FAC
:100A56002D121D80800D121C838F82758300742DCC
:100A660012086A121C8E1209A98F668E658D648C17
:100A760063757201756D00756CCA756B9A756A3B04
:100A8600E4FFFEFDFCAB6DAA6CA96BA86AD3120944
:100A9600CD5003020B26121C8EA86A1209178F71FD
:100AA6008E708D6F8C6EEC4D4E4F7004E572702318
:100AB600E5712430FFE569456845677005121D80BC
:100AC600800EAE73121C858E82758300EF12086A43
:100AD600E4F572AF6DAE6CAD6BAC6AAB71AA70A982
:100AE6006FA86E12088CCAEECAC9EDC9C8ECC8C395
:100AF600E5669FF566E5659AF565E56499F564E54D
:100B06006398F563AF6DAE6CAD6BAC6AE47B0AFAC5
:100B1600F9F81209178F6D8E6C8D6B8C6A020A8636
:100B2600E568456945676010AB67AA68A96985737A
:080B360082758300E412086AD5
:010B3E002294
:100F3500308F426831D1407433173E8034633C8C26
:100F450035B13A98370938A4386636B039C734BC54
:100F55003B2D32C83C9D30D43E0F2EE03F882CEC13
:100F650041062AF8428D29044418271045AB251C53
:100F75004741232848E121344A861F404C311D4C06
:100F85004DE21B584F9C1964515D17705323157C16
:100F950054EF138856C4119458A20FA05A830DAC70
:100FA5005C6D0BB85E6009C4605807D0625A05DCF9
:100FB500646203E8667301F4688A00006AA1FE0CA6
:100FC5006CB8FC186ECFFA2470E6F830000000000B
:10181A00F583E493FE740193FFE55925E025E02260
:10182A00F583C37401939FFFE4939EFEE4228F5ACB
:10183A008E598D588C57228F568E558D548C532223
:08184A002435F582E4340F227D
:101C9700C3EF9DEE9C400AD3EF9BEE9A50037F0162
:041CA700227F002276
:040C57008E578F58CD
:100C5B00E4F55912182312184AF583E493FC740136
:100C6B0093FD1218232439F582E4340FF583E493B2
:100C7B00FA740193FBAF58AE57121C97EF70030237
:100C8B000D4F12182312184A12181A2439F582E440
:100C9B00340F12182A8F5D8E5CF55BF55A121823F0
:100CAB00243BF582E4340F12181A2437F582E4340E
:100CBB000F12182A8F618E60F55FF55EAD5FAC5E2B
:100CCB001209A98F618E608D5F8C5EAE57AF58E4B1
:100CDB00FCFDEEC0E0EFC0E012182312184AF583BA
:100CEB00E493FE740193FBCAEECAD0E0FFD0E0FEA2
:100CFB00C3EF9BFFEE9AFEED9400FDEC9400FCAB72
:100D0B0061AA60A95FA85E12088CAB5DAA5CA95BA7
:100D1B00A85A1215D8C8ECC8C9EDC9CAEECACBEF90
:100D2B00CB1218232437F582E4340FF583E493FEBA
:100D3B00740193FFE4FCFDEB2FFFEA3EFEED39FD62
:100D4B00EC38FC220559E559C394275003020C5E7D
:050D5B00E4FFFEFDFCB9
:010D60002270
:011D8300223D
:10146400121838AB5AAA59A958A857E8C0E078A46A
:10147400E6FE08E6FFE4FCFDD0E0F812088C121842
:1014840038780E1209DE12183878A6E6FE08E6FF50
:10149400EE3395E0FDFCE55A2FF55AE5593EF55932
:1014A400E5583DF558E5573CF557AF5AAE59AD5898
:0214B400FC2218
:0214B6008D5255
:1014B800120C57121841121464121841E5521460A4
:1014C8001C14702DE47FE87E03FDFCAB56AA55A9D9
:1014D80054A85312088CE47BE87A0B800CAF56AE04
:1014E80055AD54AC53E47B03FAF9F81215D8121829
:0914F80041AF56AE55AD54AC53A2
:0115010022C7
:1010740002003EE493A3F8E493A34003F68001F254
:1010840008DFF48029E493A3F85407240CC8C3337D
:10109400C4540F4420C8834004F456800146F6DF4C
:1010A400E4800B0102040810204080900036E47EA6
:1010B400019360BCA3FF543F30E509541FFEE49341
:1010C400A360010ECF54C025E060A840B8E493A308
:1010D400FAE493A3F8E493A3C8C582C8CAC583CA33
:1010E400F0A3C8C582C8CAC583CADFE9DEE780BEEB
:0100390000C6
:10081200BB010689828A83E0225002E722BBFE02E4
:09082200E32289828A83E4932217
:10082B00BB010CE58229F582E5833AF583E0225082
:10083B0006E92582F8E622BBFE06E92582F8E222CC
:0D084B00E58229F582E5833AF583E49322E6
:10085800BB010689828A83F0225002F722BBFE017F
:02086800F32279
:10086A00F8BB010DE58229F582E5833AF583E8F0C4
:10087A00225006E92582C8F622BBFE05E92582C870
:02088A00F22258
:10088C00E88FF0A4CC8BF0A42CFCE98EF0A42CFC0B
:10089C008AF0EDA42CFCEA8EF0A4CDA8F08BF0A489
:1008AC002DCC3825F0FDE98FF0A42CCD35F0FCEBE8
:1008BC008EF0A4FEA9F0EB8FF0A4CFC5F02ECD39AD
:0F08CC00FEE43CFCEAA42DCE35F0FDE43CFC221A
:1008DB0075F008758200EF2FFFEE33FECD33CDCCD4
:1008EB0033CCC58233C5829BED9AEC99E582984057
:1008FB000CF582EE9BFEED9AFDEC99FC0FD5F0D634
:10090B00E4CEFBE4CDFAE4CCF9A88222B800C1B95D
:10091B000059BA002DEC8BF084CFCECDFCE5F0CB9B
:10092B00F97818EF2FFFEE33FEED33FDEC33FCEBD4
:10093B0033FB10D703994004EB99FB0FD8E5E4F98F
:10094B00FA227818EF2FFFEE33FEED33FDEC33FC7C
:10095B00C933C910D7059BE99A4007EC9BFCE99A70
:10096B00F90FD8E0E4C9FAE4CCFB2275F010EF2FB5
:10097B00FFEE33FEED33FDCC33CCC833C810D707B5
:10098B009BEC9AE899400AED9BFDEC9AFCE899F8F0
:0E099B000FD5F0DAE4CDFBE4CCFAE4C8F92283
:1015D800C2D5E830E70FB2D5E4C39BFBE49AFAE43E
:1015E80099F9E498F8EC30E717B2D512160E1209FB
:1015F80017E4C39BFBE49AFAE499F9E498F88003AA
:1016080012091730D50DE4C39FFFE49EFEE49DFD4B
:04161800E49CFC2230
:0E09A900C3E49FFFE49EFEE49DFDE49CFC225F
:1009B700EB9FF5F0EA9E42F0E99D42F0EC6480C8B7
:0609C70064809845F02257
:1009CD00EB9FF5F0EA9E42F0E99D42F0E89C45F080
:0109DD0022F7
:1009DE00E86010ECA2E713FCED13FDEE13FEEF132F
:0409EE00FFD8F0221C
:1009F200D083D082F8E4937012740193700DA3A394
:100A020093F8740193F5828883E4737402936860A7
:060A1200EFA3A3A380DFA7
:00000001FF
